:1000000000308A00D02900000A108A100A118207E5
:100010007E3430346D34793433345B341F3470348F
:100020007F3473340A108A100A1182074834453429
:100030004C344C344F340A34003483160611831286
:1000400006110830F80024280000F8173528F813A6
:10005000A40C03180615031C06117817352878130D
:10006000F80B28283328000006151C308400840B68
:1000700037283A28F81B2728781B2F28E229AB01BC
:100080002908AA002A08FA0000302804AC007A08DF
:10009000AD002D08AF002C08AE00831605108312AA
:1000A00005108316851083128510B00130080E3CB0
:1000B000031C7C282E080139F700FA0177087A041E
:1000C000031D642805116528051583160511031005
:1000D0008312AF0CAE0C8316851083128514B10108
:1000E0003108093C031C7628B10A70288316851054
:1000F00083128510B00A5628831605108312051442
:10010000003424308400831300080319952801303B
:10011000F800F701F70B8A28F80B89284A30F70016
:10012000F70B90289328800B8728003483168614B9
:100130008312861899280830F700A301F717AE2814
:10014000F713AE28031086180314A30C7717AE28F4
:100150007713F70BA2282308F800BA281C30F71BE6
:100160000730F800F80BB2280000F71BA028771B17
:10017000A828A2286B2A2808F80127020318C328F8
:100180002708F700CF28F7010830A900A70DF70DC1
:10019000280877020318F700F80DA90BC628FA28DB
:1001A000F701F801270803102818F707F70CF80CD7
:1001B000A818F707F70CF80C2819F707F70CF80C34
:1001C000A819F707F70CF80C281AF707F70CF80C22
:1001D000A81AF707F70CF80C281BF707F70CF80C10
:1001E000A81BF707F70CF80C01292308A7000A3011
:1001F000A800BB287808A4002408A7000A30A8009B
:10020000D02878082302A500A408031D0929A60107
:1002100022292408093C031C122924080420F80080
:10022000A600222924080A3C031D19297E30A600B5
:10023000222924080B3C031D20293630A600222940
:100240004F30A60025080420A7002608A80027088C
:10025000A9003F20742AA401A30124084E3C031CDA
:100260004129031D372923081F3C031C41298618F7
:100270003C290130F80043290000A30A0319A40A0D
:100280002D290030F8000034A801A9013F202B21BE
:10029000F808031D8129A8016730A9003F202B2100
:1002A000F808031D81296730A8003E30A9003F20CF
:1002B0002B21F808031D81293E30A8005B30A900DE
:1002C0003F202B21F808031D81295B30A800A900DD
:1002D0003F202B21F808031D81295B30A8003B300B
:1002E000A9003F202B21F808031D81293B30A800DD
:1002F000A9013F202B21F808031D8129A801A9018C
:100300003F20BD2AA801A9013F202B21F808031D89
:10031000CF29A8011F30A9003F202B21F808031D79
:10032000CF291F30A8007730A9003F202B21F808E3
:10033000031DCF297730A8003D30A9003F202B2195
:10034000F808031DCF293D30A800A9013F202B212B
:10035000F808031DCF29A8017730A9003F202B21E1
:10036000F808031DCF297730A8005B30A9003F2093
:100370002B21F808031DCF295B30A800A9003F20DE
:100380002B21F808031DCF295B30A800A9013F20CD
:100390002B21F808031DCF29A801A9013F20C22A5B
:1003A000840183131F3083058316061183120615FB
:1003B00007309F00A101A30123081220A30AF70020
:1003C000A4001D2806302302031DDC298316861491
:1003D0008312A801A9013F200230A300C830A40065
:1003E0008120A30BEE29A8015B30A9003F20023039
:1003F000A300C830A4008120A30BF9295B30A8001A
:100400003E30A9003F200230A300C830A400812064
:10041000A30B052A3E30A8006730A9003F20023018
:10042000A300C830A4008120A30B112A6730A800C4
:10043000A9013F200230A300C830A4008120A30BF3
:100440001C2AA8011F30A9003F200230A300C83099
:10045000A4008120A30B272A1F30A8003030A90058
:100460003F200230A300C830A4008120A30B332A10
:100470003030A8000F30A9003F200230A300C83060
:10048000A4008120A30B3F2A0F30A8000D30A90043
:100490003F200230A300C830A4008120A30B4B2AC8
:1004A0000D30A8001730A9003F200230A300C8304B
:1004B000A4008120A30B572A1730A800A9013F20D0
:1004C0000230A300C830A4008120A30B622AA80137
:1004D000A9013F2096287808A2002208773C031C37
:1004E000742A2208A300F5282208F03C031D7B2A69
:1004F000A801A9013F202208F13C031D832A0130F5
:10050000A800A9003F202208F23C031D8B2A4F308F
:10051000A800A9003F202208F33C031D942A1330B1
:10052000A8002530A9003F202208F43C031D9D2A85
:100530004730A8003E30A9003F202208F53C031DAB
:10054000A62A1D30A8005B30A9003F202208F63CF7
:10055000031DAF2A1F30A8007730A9003F202208D2
:10056000F73C031DB82A1730A8003030A9003F20FF
:100570002208F83C031DBD2A44292208F93C031D2A
:10058000C22A82292208FA3C031DCB2A6D30A8001A
:100590003030A9003F202208FB3C031DD42A6D30D7
:1005A000A8007E30A9003F202208FC3C031DDD2A64
:1005B0007E30A8003030A9003F202208FD3C031DFA
:1005C000E52A7E30A800A9003F202208EE3C031D4A
:1005D000EE2A4F30A8003030A9003F202208EF3C1F
:1005E000031DF72A4F30A8006D30A9003F206A2A6A
:0205F0006300A6
:02400E00213F50
:00000001FF
